:0200000480007A
:10000000971700009387070093001000130100006A
:10001000B701F17F9381F1FF370200809302F0FF77
:1000200073900234F3B00034F3900234733101342E
:1000300073910234F3B10134F39102347332023418
:1000400073920234F3B20234F312003423A0070097
:1000500023A2170023A4270023A6370023A84700C4
:1000600023AA570097120000938242FB93051000C9
:1000700013060000B706F17F9386F6FF370700806E
:100080009307F0FF73900734F3B5053473360634E5
:10009000F3B6063473370734F3B7073473380034D4
:1000A00023A0B20023A2C20023A4D20023A6E20010
:1000B00023A8F20023AA0201171D0000130D8DF7DB
:1000C000B75A3412938A8A67130AF0FF73100A34FE
:1000D00073BB0A34F33A0B34F31B0A3473BC0B348E
:1000E000F33C003423205D0123226D0123247D0194
:1000F00023268D0123289D01971000009380C0F4D2
:10010000377F7242130FFFE673100F3473300F34D2
:1001100023A0000023A2E00117110000130141F306
:10012000B79FFFF7938F8F8173900F347330003434
:1001300073300034F33F0034232001002322F10107
:1001400017110000130141F11302F0FFB752389666
:1001500093824227B7531632938383497310023434
:10016000F3B20234F3B30334733404342320510064
:10017000232271002324810017150000130585E850
:1001800097150000938505EE370610F01306C6F2AA
:100190006306B5028326C5002320D600832685008A
:1001A0002320D600832645002320D6008326050081
:1001B0002320D600130505016FF09FFD370510F0D1
:1001C000130505F2232005000000000000000000D8
:0401D000000000002B
:10100000FFFFFFFFFFFFFFFFFFFFFFFFFFFFFFFFF0
:10101000FFFFFFFFFFFFFFFFFFFFFFFFFFFFFFFFE0
:10102000FFFFFFFFFFFFFFFFFFFFFFFFFFFFFFFFD0
:10103000FFFFFFFFFFFFFFFFFFFFFFFFFFFFFFFFC0
:10104000FFFFFFFFFFFFFFFFFFFFFFFFFFFFFFFFB0
:10105000FFFFFFFFFFFFFFFFFFFFFFFFFFFFFFFFA0
:040000058000000077
:00000001FF
